:02000000932843
:080008004328820750344934FB
:1000100043342D3441344434433420345634323460
:100020002E34303431340D340A34003450344934F1
:1000300043342D344C344F34473420345634313427
:100040002E34303430340D340A34003450344934D2
:1000500043342D345234453441344C3456343134E5
:100060002E34303430340D340A3400348207803476
:10007000403420341034A80803193B28A801A808EC
:10008000031D3E280800A000030E8301A3000408FE
:10009000A10084010A08A2008A018B1860280B19AC
:1000A0007B2856282408A900FF30A80022088A00CF
:1000B00021088400230E8300A00E200E8B1009005F
:1000C0002B08A600A60B62280830A5002C08A60065
:1000D000A60B6828061C031006180314A40CA50B15
:1000E00066282D08A600A60B73282D08A600A60BCF
:1000F00077288B1052284F3081000B110130BB0242
:10010000031CBC02031CBD02031CBE0203185628BC
:100110004E08BB004F08BC005008BD005108BE008F
:10012000E130AA0056288316183081008312850119
:100130000730860083161F308500F1308600831259
:100140004F30AB00AA30AC005530AD00AA30AE0045
:10015000AA30AF00AA30B000A801AA017623762306
:10016000762390308B00BB01BC01BD01BE01BF01F5
:10017000482241304A02031DC52844304B02031D6A
:10018000C528CC1FC5280130BF008A013F0882075F
:10019000CD284029F928BF01C5288B128B1ACD28FC
:1001A0003B203F3029020319E42A2908B1005723D4
:1001B000613029020319122A673029020319352AEE
:1001C000643029020319F5297230290203196C2AB7
:1001D000773029020319B62A693029020319C02988
:1001E0006F3029020319C929733029020319D12953
:1001F000C5288B138B1BF92830308B008B17A80870
:10020000031913293B203F3029020319E92A290841
:10021000B10057238B128B1A0A2974302902031D4F
:10022000C528BF01C528AA080319C528CD1F1E2946
:1002300000309F007C211E08B10057234D1F262946
:1002400008309F007C211E08B1005723CD1E2E29A7
:1002500010309F007C211E08B10057234D1E362907
:1002600018309F007C211E08B10057237721C52834
:10027000C1309F007C211E08B10057237721C5287B
:100280008B138B1B402930308B008B17A808031968
:100290005A293B203F3029020319E62A2908B100D8
:1002A00057238B128B1A512974302902031DC5283C
:1002B000BF01C528AA080319C528CD1F632901302D
:1002C0009F007C218D214D1F692909309F007C21D1
:1002D0008D21CD1E6F2911309F007C218D214D1E57
:1002E000752919309F007C218D217721C528AA010D
:1002F000AA08031D772908004D0883169F00831262
:100300004D08C800C80EC030C805481448089F04EE
:1003100076231F151F198A290800482241304A02F6
:10032000031DBD2944304B02031DBD29CC1FBD292F
:100330005608B8005708B7001E08B400A6220130BE
:10034000D6070318D70755085702031CB1295608CA
:1003500054020318B1294C1BBE295208D600530879
:10036000D700B7010C30B8005608B400A622B70178
:100370000D30B8005708B400A6220800BF010800DD
:100380008316F1308600831200000608B10057235F
:10039000C5283B2083160130860083122908860079
:1003A000C5280630B200E621031DC5285330B10030
:1003B00057234108AB004208AC004308AD00440895
:1003C000AE004508AF004608B000C52841308400A3
:1003D000C7013B202908C70729088000840AB20BFF
:1003E000E9293B202908C70708000530B200E621AB
:1003F000031DC5284430B10057234108CD004208F1
:10040000CE004308CF004408D0004508D1004E0874
:10041000BB004F08BC005008BD005108BE000230B0
:10042000BF00C5280330B200E621031DC5284130B6
:10043000B1005723831641089F008312FC30C10589
:10044000411441089F004208BA004308B9009E01C8
:100450001E08B1001F1557231F192C2A0130BA029C
:10046000031CB9020318282AC5283B208316290833
:100470009F008312FC30A905291429089F004122FE
:10048000C5281F151F19422A1E08B100572308004E
:10049000B701B801B9010D30BA004A308400FE221C
:1004A000A030B6000E233708B6000E233808B60079
:1004B0000E23FE22A130B6000E232D233408800027
:1004C000840A0130BA020130031CB902031C692AF4
:1004D0005D2A3423072308000430B200E621031DFF
:1004E000C5284108B8004208B7004308BA004408CC
:1004F000B9005230B10057230130BA02031CB902CF
:10050000FE22A030B6000E233708B6000E233808AE
:10051000B6000E23FE22A130B6000E232D23340890
:10052000B10057233B2029083402031DA42A0130BF
:10053000BA02031CB90203188E2A34230723340895
:10054000B10057233B20C5280723C528F622FE22E9
:10055000A030B6000E233708B6000E233808B600C8
:100560000E233408B6000E23072308000430B2001F
:10057000E621031DC5284108B8004208B70043081A
:10058000BA004408B9005730B1005723FE22A0300A
:10059000B6000E233708B6000E233808B6000E2327
:1005A0003B202908B6000E230723F6222908B100B4
:1005B00057230130B8070318B7070130BA02031CEC
:1005C000B9020318C62AC528C001EB2A1030C000A2
:1005D000EB2A2030C0008A011030C70040080520F7
:1005E000B1005723C00AC70BEE2AC528FE22A0304F
:1005F000B6000E2307233618F62A08008615522364
:10060000061552238611522306115223080006159F
:100610005223861552230611522308000830B500D4
:10062000B60D031C86110318861552230615522396
:100630000611B50B102B8316F93086008312522356
:1006400006157623B6018619B6038316F1308600A7
:10065000831206115223861108003B2386110615CA
:1006600052230611522308003B23861506155223F8
:100670000611522308000830B5008316F9308600B1
:10068000831206155223861D031086190314B40D18
:1006900006115223B50B412B8316F13086008312CD
:1006A00052230800532B542B552B562B08008B1329
:1006B0008B1B572B86102E08B300B30B5D2B083015
:1006C000B200B10C031C8610031886142F08B30067
:1006D000B30B682BB20B612B6D2B6E2B6F2B86141B
:1006E0008B173008B300B30B732B08001330C8000E
:1006F0005B30C9000000000000000000C90B7A2B2D
:06070000C80B782B080075
:02400E00723FFF
:00000001FF
